:020000000628D0
:080008000B110900831685109D
:1000100083120130A5000C216F200130A5000C21B6
:100020000130003C031940282030A700803027020F
:10003000013003180001003C03193F2827089100F4
:100040004F200030A1000530A200FC2027089300BB
:1000500076200030A1000A30A200FC20270895007D
:10006000A3200130A1000230A200FC202708970045
:10007000CF200130A5000C216F20A70A16281028D8
:100080000E0890006E308F0000000000000000009D
:10009000000000008F0B4428900B422808008510B8
:1000A000FF3092001208003C013003190001920356
:1000B000003C03195C2852280930031003188510EE
:1000C000031C85146328103E031C6228FF3E910C1C
:1000D000031D5E2885100A308E0040200800FE3087
:1000E00091004F20013091004F2008000030940013
:1000F0001308633C013003180001003C03198628F3
:100100006430130293001408940A782830301407DE
:1001100091004F20003094001308093C013003186F
:100120000001003C03199A280A30130293001408B6
:10013000940A8C283030140791004F203030130778
:1001400091004F2008001508F0399600960E0A30ED
:100150001602013003180001003C0319B4283030A6
:10016000160791004F20B9280A301602413E91002F
:100170004F2015080F3996000A3016020130031877
:100180000001003C0319C9283030160791004F20A8
:10019000CE280A301602413E91004F2008008030E0
:1001A00098004030990020309A0010309B000830B1
:1001B0009C0004309D0002309E0001309F00003002
:1001C000A00008302002013003180001003C031990
:1001D000FB282008183E840000081705003C03197E
:1001E000F528313091004F20F828303091004F2011
:1001F0002008A00AE1280800FE3091004F208C0161
:1002000021088D0040308C078D0B02290C08803EA0
:10021000220791004F2008000030A6000A30260275
:10022000013003180001003C03191B2964308E00C3
:080230004020A60A0E29080077
:00000001FF
